:100000000C942A000C9445000C9445000C94450077
:100010000C9445000C9445000C9445000C9445004C
:100020000C9445000C9445000C9445000C9445003C
:100030000C9445000C9445000C9445000C9445002C
:100040000C9445000C9445000C9445000C9445001C
:100050000C94450011241FBECFE5D4E0DEBFCDBF18
:1000600010E0A0E6B0E0E2EFF1E002C005900D92F2
:10007000A236B107D9F710E0A2E6B0E001C01D92A8
:10008000A236B107E1F70C94D1000C940000CF9395
:10009000DF93CDB7DEB781E0809338001092350052
:1000A0001092320081E08093370010923400109259
:1000B0003100DF91CF910895CF93DF93CDB7DEB7B5
:1000C00025970FB6F894DEBF0FBECDBF8983898117
:1000D000282F33273D832C838C819D81813091058E
:1000E000B9F02C813D81223031052CF48C819D8129
:1000F000009739F03AC02C813D812230310571F0F2
:1001000034C08EEF9091380089238093380040C02E
:10011000809138008160809338003AC09EEF8091D2
:10012000380089238093380080E29EE49B838A8391
:100130008A819B81009731F08A819B8101979B8303
:100140008A83F6CF8091380081608093380080E206
:100150009EE49B838A838A819B810097C9F08A8170
:100160009B8101979B838A83F6CF809136009927E4
:1001700081709070009739F08EEF9091380089234C
:100180008093380005C080913800816080933800EA
:1001900025960FB6F894DEBF0FBECDBFDF91CF918D
:1001A0000895CDE5D4E0DEBFCDBF0E94470080E0DA
:1001B0000E945C0080E69AEE9A83898389819A8105
:1001C000009731F089819A8101979A838983F6CFCC
:1001D00081E00E945C0080E69AEE9A83898389819F
:1001E0009A81009721F389819A8101979A83898363
:0201F000F6CF48
:0201F20001000A
:00000001FF
